:100000000206E67DA37C08ED1D70011C144C70F700
:0A001000EF1F70011E144E70EA226B
:1000230002064BEFD394077480948040037FFF2232
:1000330012029DFED394037480948040037FFF22B9
:10004300EF7044EE700B9000011202B6F45293521B
:100053009412029D6401700B9000011202B6429348
:10006300F4529412029DFE6402700A90000112027F
:10007300B642934294EE6403700D9000011202B6EF
:10008300FEF45293EE4294EF6401704612029DFE19
:10009300700B9000011202B6F452915292EE640179
:1000A300700B9000011202B64291F4529212029D1B
:1000B3006402700A9000011202B642914292120247
:1000C3009D6403700D9000011202B6FEF45291EE8E
:1000D3004292EF6402704612029DFE700B90000183
:1000E3001202B6F452955296EE6401700B90000121
:1000F3001202B64295F4529612029D6402700A905F
:1001030000011202B64295429612029D6403700DDD
:100113009000011202B6FEF45295EE4296EF64038C
:10012300704612029DFE700B9000011202B6F4524B
:10013300B152B2EE6401700B9000011202B642B1EB
:10014300F452B212029D6402700A9000011202B6C8
:1001530042B142B212029D6403700D90000112027B
:10016300B6FEF452B1EE42B2EF6404704612029D41
:10017300FE700B9000011202B6F452B352B4EE6457
:1001830001700B9000011202B642B3F452B4120292
:100193009D6402700A9000011202B642B342B41287
:1001A300029D6403700D9000011202B6FEF452B377
:1001B300EE42B4EF6405704612029DFE700B900090
:1001C300011202B6F452C952CAEE6401700B9000D8
:1001D300011202B642C9F452CA12029D6402700AA5
:1001E3009000011202B642C942CA12029D64037012
:1001F3000D9000011202B6FEF452C9EE42CAEF643A
:1002030006704612029DFE700B9000011202B6F4B6
:1002130052CB52CCEE6401700B9000011202B64235
:10022300CBF452CC12029D6402700A9000011202B8
:10023300B642CB42CC12029D6403700D90000112B2
:1002430002B6FEF452CBEE42CCEF640770491202C1
:100253009DFF7E00700B9000011202B6F452E15232
:10026300E2EF64014E700B9000011202B642E1F41A
:1002730052E212029D6402700A9000011202B64219
:10028300E142E212029D6403700D9000011202B676
:10029300FFF452E1EF42E27F0022BB010689828A2A
:1002A30083E0225002E722BBFE02E32289828A8393
:1002B300E49322BB010CE58229F582E5833AF583B9
:1002C300E0225006E92582F8E622BBFE06E92582F4
:1002D300F8E222E58229F582E5833AF583E4932265
:1002E30075F008758200EF2FFFEE33FECD33CDCCD2
:1002F30033CCC58233C5829BED9AEC99E582984055
:100303000CF582EE9BFEED9AFDEC99FC0FD5F0D631
:10031300E4CEFBE4CDFAE4CCF9A88222B800C1B95B
:100323000059BA002DEC8BF084CFCECDFCE5F0CB99
:10033300F97818EF2FFFEE33FEED33FDEC33FCEBD2
:1003430033FB10D703994004EB99FB0FD8E5E4F98D
:10035300FA227818EF2FFFEE33FEED33FDEC33FC7A
:10036300C933C910D7059BE99A4007EC9BFCE99A6E
:10037300F90FD8E0E4C9FAE4CCFB2275F010EF2FB3
:10038300FFEE33FEED33FDCC33CCC833C810D707B3
:100393009BEC9AE899400AED9BFDEC9AFCE899F8EE
:1003A3000FD5F0DAE4CDFBE4CCFAE4C8F922EB9FF5
:1003B300F5F0EA9E42F0E99D42F0E89C45F022E820
:1003C300600FECC313FCED13FDEE13FEEF13FFD828
:1003D300F122BB010DE58229F582E5833AF583021B
:1003E30004125007E92582F8020405BBFE07E9253C
:1003F30082F802041EE58229F582E5833AF5830239
:10040300042BE6FB08E6F908E6FA08E6CBF822E057
:10041300F8A3E0F9A3E0FAA3E0FB22E2FB08E2F988
:1004230008E2FA08E2CBF822E493F8740193F97432
:100433000293FA740393FB228B128A138914EF64D9
:100443000160030205A4751901F51AF51BF51CF5E6
:100453001DF51EF51FFFEFC3948074809480500F29
:1004630074802FF582E43400F583E4F00F80E7E431
:10047300FFEFC3948074809480500F74002FF58233
:10048300E43400F583E4F00F80E7AB12AA13A91458
:1004930012029DFFE598543F4FF598EF64C0600842
:1004A300EF644060030205539000021203D57F00FE
:1004B3007E607D547C0012031F8F188E178D168C5F
:1004C30015E4FFFE7D01FCAB18AA17A916A815C3F6
:1004D3001203B140037FFF22C3E49518F518E49596
:1004E30017F51774019516F516E49515F515AB1266
:1004F300AA13A9149000011202B664027026538E47
:10050300EF438E01538EF7438E04AF18AE17AD162B
:10051300AC1578081203C28FD68518D753AFFB43A7
:100523008E108066C28E538EFE5389BF5389CF438C
:100533008E40AF18AE17AD16AC1578081203C28FF4
:100543008D85188BC2AB5389BF538FFDD28E803AF2
:10055300AB12AA13A91412029DFF7E00701490001F
:10056300081202B664017005438E20801D538EDF8E
:100573008018EF64804E70129000081202B6640176
:100583007005438780800353877FAB12AA13A91496
:100593009000071202B67004C29C8002D29C7F00B6
:1005A300227FFF221206D6120696D2AF7BFF7A066F
:1005B30079FC1206C37F017E00120003D3E51E946B
:1005C300007480948040EE151EE51E70E8D3E51D8F
:1005D300940074809480401EE4F508E508C3951DDB
:1005E300501474002508F582E43400F583E0FF120B
:1005F30006F2050880E5E4F51D80BAEFFBD394010C
:10060300748094805009EB7004C2AC8002D2ACEDCC
:10061300FF7E00D39403748094805029EF700553B8
:10062300B7EFC2BCEF64014E700553B7EFD2BCEF16
:1006330064024E700543B710C2BCEF64034E7005ED
:1006430043B710D2BC7F0022C0E0C083C082C0D0B9
:1006530075D000C007309828C298E51F7022C3E503
:100663001D9480748094804003751D00AF1D051D8B
:1006730074002FF582E43400F583E599F0751E05C7
:10068300309905C299751C00D007D0D0D082D08391
:10069300D0E032750940750A01750E00750DC275FB
:1006A3000C01750B00751001E4F511FB7A00790953
:1006B3007F0112043B7D017F011205FE53A23F22FD
:1006C30012029DFF600C1206F2740129F9E43AFA52
:1006D30080EE22750A03E4F509FB7A0079097F03AA
:1006E300020026787FE4F6D8FD75811F0205A78FE7
:1006F30099751C01E51C70FC225354433820554165
:1007030052543120546573742050726F6772616D57
:060713006D65210D0A00D6
:00000001FF
